******************************************************************************
                  TI ARM Linker PC v5.1.0                      
******************************************************************************
>> Linked Wed Sep 04 08:45:52 2013

OUTPUT FILE NAME:   <TMS570LS3137_Test_CAN_TX.out>
ENTRY POINT SYMBOL: "_c_int00"  address: 00005bc8


MEMORY CONFIGURATION

         name            origin    length      used     unused   attr    fill
----------------------  --------  ---------  --------  --------  ----  --------
  VECTORS               00000000   00000020  00000020  00000000     X
  FLASH0                00000020   0017ffe0  00006670  00179970  R  X
  FLASH1                00180000   00180000  00000000  00180000  R  X
  STACKS                08000000   00001500  00000000  00001500  RW  
  RAM                   08001500   0003eb00  00000018  0003eae8  RW  


SEGMENT ALLOCATION MAP

run origin  load origin   length   init length attrs members
----------  ----------- ---------- ----------- ----- -------
00000000    00000000    00006690   00006690    r-x
  00000000    00000000    00000020   00000020    r-x .intvecs
  00000020    00000020    00006414   00006414    r-x .text
  00006434    00006434    00000224   00000224    r-- .const
  00006658    00006658    00000038   00000038    r-- .cinit
08001500    08001500    00000018   00000000    rw-
  08001500    08001500    00000010   00000000    rw- .data
  08001510    08001510    00000008   00000000    rw- .bss


SECTION ALLOCATION MAP

 output                                  attributes/
section   page    origin      length       input sections
--------  ----  ----------  ----------   ----------------
.intvecs   0    00000000    00000020     
                  00000000    00000020     sys_intvecs.obj (.intvecs)

.text      0    00000020    00006414     
                  00000020    000026ec     sys_selftest.obj (.text)
                  0000270c    00000adc     system.obj (.text)
                  000031e8    00000874     sys_vim.obj (.text)
                  00003a5c    0000085c     can.obj (.text)
                  000042b8    0000065c     rti.obj (.text)
                  00004914    00000630     pinmux.obj (.text)
                  00004f44    00000620     esm.obj (.text)
                  00005564    000003c4     sys_core.obj (.text)
                  00005928    000002a0     sys_vim.obj (.text:retain)
                  00005bc8    00000248     sys_startup.obj (.text:retain)
                  00005e10    00000158     esm.obj (.text:retain)
                  00005f68    00000110     notification.obj (.text)
                  00006078    000000e8     dabort.obj (.text)
                  00006160    0000009c     rtsv7R4_T_be_v3D16_eabi.lib : memcpy_t2.obj (.text)
                  000061fc    00000094                                 : auto_init.obj (.text)
                  00006290    00000060                                 : copy_decompress_rle.obj (.text)
                  000062f0    0000004c     rti.obj (.text:retain)
                  0000633c    00000048     rtsv7R4_T_be_v3D16_eabi.lib : cpy_tbl.obj (.text)
                  00006384    00000044                                 : exit.obj (.text)
                  000063c8    0000002c     sys_main.obj (.text)
                  000063f4    00000014     rtsv7R4_T_be_v3D16_eabi.lib : _lock.obj (.text)
                  00006408    00000012                                 : copy_zero_init.obj (.text:decompress:ZI)
                  0000641a    0000000e                                 : copy_decompress_none.obj (.text:decompress:none)
                  00006428    00000006                                 : copy_decompress_rle.obj (.text:decompress:rle24)
                  0000642e    00000002     --HOLE-- [fill = 0]
                  00006430    00000004     sys_phantom.obj (.text:retain)

.const     0    00006434    00000224     
                  00006434    00000204     sys_vim.obj (.const:s_vim_init)
                  00006638    00000020     can.obj (.const)

.cinit     0    00006658    00000038     
                  00006658    00000011     (.cinit..data.load) [load image, compression = rle]
                  00006669    00000003     --HOLE-- [fill = 0]
                  0000666c    0000000c     (__TI_handler_table)
                  00006678    00000008     (.cinit..bss.load) [load image, compression = zero_init]
                  00006680    00000010     (__TI_cinit_table)

.data      0    08001500    00000010     UNINITIALIZED
                  08001500    00000008     rtsv7R4_T_be_v3D16_eabi.lib : _lock.obj (.data)
                  08001508    00000008                                 : exit.obj (.data)

.bss       0    08001510    00000008     UNINITIALIZED
                  08001510    00000008     (.common:Tx_Data_CAN)


LINKER GENERATED COPY TABLES

__TI_cinit_table @ 00006680 records: 2, size/record: 8, table size: 16
	.data: load addr=00006658, load size=00000011 bytes, run addr=08001500, run size=00000010 bytes, compression=rle
	.bss: load addr=00006678, load size=00000008 bytes, run addr=08001510, run size=00000008 bytes, compression=zero_init


LINKER GENERATED HANDLER TABLE

__TI_handler_table @ 0000666c records: 3, size/record: 4, table size: 12
	index: 0, handler: __TI_zero_init
	index: 1, handler: __TI_decompress_rle24
	index: 2, handler: __TI_decompress_none


GLOBAL SYMBOLS: SORTED ALPHABETICALLY BY Name 

address    name
--------   ----
00006385   C$$EXIT
00004644   IsdwdKeySequenceCorrect
UNDEFED    SHT$$INIT_ARRAY$$Base
UNDEFED    SHT$$INIT_ARRAY$$Limit
08001510   Tx_Data_CAN
00006680   __TI_CINIT_Base
00006690   __TI_CINIT_Limit
0000666c   __TI_Handler_Table_Base
00006678   __TI_Handler_Table_Limit
00005920   __TI_PINIT_Base
00005924   __TI_PINIT_Limit
000061fd   __TI_auto_init
08001508   __TI_cleanup_ptr
0000641b   __TI_decompress_none
00006429   __TI_decompress_rle24
0800150c   __TI_dtors_ptr
00000000   __TI_static_base__
00006409   __TI_zero_init
00006161   __aeabi_memcpy
00006161   __aeabi_memcpy4
00006161   __aeabi_memcpy8
ffffffff   __binit__
ffffffff   __c_args__
00005bc8   _c_int00
00005818   _coreClearAuxiliaryDataFault_
00005834   _coreClearAuxiliaryInstructionFault_
000057e0   _coreClearDataFaultAddress_
000057a8   _coreClearDataFault_
000057fc   _coreClearInstructionFaultAddress_
000057c4   _coreClearInstructionFault_
0000570c   _coreDisableEventBusExport_
00005770   _coreDisableFlashEcc_
0000573c   _coreDisableRamEcc_
000056f4   _coreEnableEventBusExport_
00005754   _coreEnableFlashEcc_
00005788   _coreEnableIrqVicOffset_
00005724   _coreEnableRamEcc_
000056dc   _coreEnableVfp_
00005810   _coreGetAuxiliaryDataFault_
0000582c   _coreGetAuxiliaryInstructionFault_
000057d8   _coreGetDataFaultAddress_
000057a0   _coreGetDataFault_
000057f4   _coreGetInstructionFaultAddress_
000057bc   _coreGetInstructionFault_
00005564   _coreInitRegisters_
00005670   _coreInitStackPointer_
00006078   _dabort
00005850   _disable_FIQ_interrupt_
00005858   _disable_IRQ_interrupt_
00005848   _disable_interrupt_
00005860   _enable_interrupt_
000058f0   _errata_CORTEXR4_57_
00005908   _errata_CORTEXR4_66_
00005868   _esmCcmErrorsClear_
000056bc   _getCPSRValue_
000056c4   _gotoCPUIdle_
08001500   _lock
00006403   _nop
000063fb   _register_lock
000063f5   _register_unlock
08001504   _unlock
00006389   abort
0000116c   adc1ParityCheck
00001228   adc2ParityCheck
ffffffff   binit
000040e4   can1GetConfigValue
00001304   can1ParityCheck
000013e0   can2ParityCheck
000014b8   can3ParityCheck
00003fb4   canDisableErrorNotification
0000400c   canDisableloopback
00003f94   canEnableErrorNotification
00003fd4   canEnableloopback
00006034   canErrorNotification
00003ce0   canGetData
00003f70   canGetErrorLevel
00003f4c   canGetLastError
00003a5c   canInit
000040c8   canIoRxGetBit
0000403c   canIoSetDirection
00004074   canIoSetPort
000040ac   canIoTxGetBit
00003ef0   canIsMessageBoxValid
00003e94   canIsRxMessageArrived
00003e38   canIsTxMessagePending
00006048   canMessageNotification
00003bf0   canTransmit
00000030   ccmSelfCheck
000025ec   ccmr4GetConfigValue
00000884   checkB0RAMECC
00000a38   checkB1RAMECC
00001b3c   checkClockMonitor
00000bec   checkFlashECC
00001c08   checkFlashEEPROMECC
00001da0   checkPLL1Slip
00001e8c   checkPLL2Slip
00001f50   checkRAMAddrParity
00001920   checkRAMECC
00002034   checkRAMUERRTest
000006e0   checkefcSelfTest
0000633d   copy_in
00000234   cpuSelfTest
00000cd0   cpuSelfTestFail
00000cc8   custom_dabort
0000605c   dmaGroupANotification
00000d94   dmaParityCheck
000046ac   dwdClearFlag
000045e0   dwdCounterEnable
00004628   dwdGenerateSysReset
00004678   dwdGetStatus
000046bc   dwdGetViolationStatus
00004564   dwdInit
0000460c   dwdReset
000045f0   dwdSetPreload
000045d4   dwwdGetCurrentDownCounter
0000458c   dwwdInit
00000590   efcCheck
00002550   efcGetConfigValue
000006b8   efcSelfTest
000005f4   efcStuckZeroTest
000050f4   esmActivateNormalOperation
000051e0   esmClearStatus
00005220   esmClearStatusBuffer
000050b8   esmDisableError
00005130   esmDisableInterrupt
0000508c   esmEnableError
00005104   esmEnableInterrupt
00005340   esmEnterSelfTest
00005070   esmError
00005404   esmGetConfigValue
0000526c   esmGetStatus
000052e0   esmGetStatusBuffer
00005f68   esmGroup1Notification
00005f78   esmGroup2Notification
00005e10   esmHighInterrupt
00004f44   esmInit
000053b4   esmSelfTestStatus
0000524c   esmSetCounterPreloadValue
0000515c   esmSetInterruptLevel
000050e4   esmTriggerErrorPinReset
00006391   exit
00002160   fmcBus1ParityCheck
000007a8   fmcBus2Check
000007e4   fmcECCcheck
00000e54   het1ParityCheck
00000fd4   het2ParityCheck
00000f08   htu1ParityCheck
00001094   htu2ParityCheck
000063c8   main
00002848   mapClocks
00006161   memcpy
00000174   memoryInit
00005f88   memoryPort0TestFailNotification
00005fa4   memoryPort1TestFailNotification
000015a4   mibspi1ParityCheck
000016b8   mibspi3ParityCheck
000017ec   mibspi5ParityCheck
00004914   muxInit
00002288   pbistFail
00002360   pbistGetConfigValue
000004dc   pbistIsTestCompleted
000004f8   pbistIsTestPassed
00000534   pbistPortTestStatus
000003e0   pbistRun
000002b4   pbistSelfCheck
000004ac   pbistStop
000027f4   periphInit
00006430   phantomInterrupt
00004c98   pinmuxGetConfigValue
00000000   resetEntry
000062f0   rtiCompare0Interrupt
0000476c   rtiDisableNotification
00004744   rtiEnableNotification
00004788   rtiGetConfigValue
000044d8   rtiGetCurrentTick
000044b0   rtiGetPeriod
000042b8   rtiInit
00005fc0   rtiNotification
00004404   rtiResetCounter
00004488   rtiSetPeriod
000043ac   rtiStartCounter
000043d8   rtiStopCounter
00000020   selftestFailNotification
000027b4   setupFlash
0000270c   setupPLL
00002fd4   sramGetConfigValue
000024b0   stcGetConfigValue
000001b8   stcSelfCheck
00000ccc   stcSelfCheckFail
00002a14   systemGetConfigValue
00002954   systemInit
000029e0   systemPowerDown
00002e28   tcmflashGetConfigValue
0000276c   trimLPO
000032a4   vimChannelMap
00003498   vimDisableInterrupt
00003340   vimEnableInterrupt
0000351c   vimGetConfigValue
000031e8   vimInit
00000cd4   vimParityCheck
00005928   vimParityErrorHandler


GLOBAL SYMBOLS: SORTED BY Symbol Address 

address    name
--------   ----
00000000   __TI_static_base__
00000000   resetEntry
00000020   selftestFailNotification
00000030   ccmSelfCheck
00000174   memoryInit
000001b8   stcSelfCheck
00000234   cpuSelfTest
000002b4   pbistSelfCheck
000003e0   pbistRun
000004ac   pbistStop
000004dc   pbistIsTestCompleted
000004f8   pbistIsTestPassed
00000534   pbistPortTestStatus
00000590   efcCheck
000005f4   efcStuckZeroTest
000006b8   efcSelfTest
000006e0   checkefcSelfTest
000007a8   fmcBus2Check
000007e4   fmcECCcheck
00000884   checkB0RAMECC
00000a38   checkB1RAMECC
00000bec   checkFlashECC
00000cc8   custom_dabort
00000ccc   stcSelfCheckFail
00000cd0   cpuSelfTestFail
00000cd4   vimParityCheck
00000d94   dmaParityCheck
00000e54   het1ParityCheck
00000f08   htu1ParityCheck
00000fd4   het2ParityCheck
00001094   htu2ParityCheck
0000116c   adc1ParityCheck
00001228   adc2ParityCheck
00001304   can1ParityCheck
000013e0   can2ParityCheck
000014b8   can3ParityCheck
000015a4   mibspi1ParityCheck
000016b8   mibspi3ParityCheck
000017ec   mibspi5ParityCheck
00001920   checkRAMECC
00001b3c   checkClockMonitor
00001c08   checkFlashEEPROMECC
00001da0   checkPLL1Slip
00001e8c   checkPLL2Slip
00001f50   checkRAMAddrParity
00002034   checkRAMUERRTest
00002160   fmcBus1ParityCheck
00002288   pbistFail
00002360   pbistGetConfigValue
000024b0   stcGetConfigValue
00002550   efcGetConfigValue
000025ec   ccmr4GetConfigValue
0000270c   setupPLL
0000276c   trimLPO
000027b4   setupFlash
000027f4   periphInit
00002848   mapClocks
00002954   systemInit
000029e0   systemPowerDown
00002a14   systemGetConfigValue
00002e28   tcmflashGetConfigValue
00002fd4   sramGetConfigValue
000031e8   vimInit
000032a4   vimChannelMap
00003340   vimEnableInterrupt
00003498   vimDisableInterrupt
0000351c   vimGetConfigValue
00003a5c   canInit
00003bf0   canTransmit
00003ce0   canGetData
00003e38   canIsTxMessagePending
00003e94   canIsRxMessageArrived
00003ef0   canIsMessageBoxValid
00003f4c   canGetLastError
00003f70   canGetErrorLevel
00003f94   canEnableErrorNotification
00003fb4   canDisableErrorNotification
00003fd4   canEnableloopback
0000400c   canDisableloopback
0000403c   canIoSetDirection
00004074   canIoSetPort
000040ac   canIoTxGetBit
000040c8   canIoRxGetBit
000040e4   can1GetConfigValue
000042b8   rtiInit
000043ac   rtiStartCounter
000043d8   rtiStopCounter
00004404   rtiResetCounter
00004488   rtiSetPeriod
000044b0   rtiGetPeriod
000044d8   rtiGetCurrentTick
00004564   dwdInit
0000458c   dwwdInit
000045d4   dwwdGetCurrentDownCounter
000045e0   dwdCounterEnable
000045f0   dwdSetPreload
0000460c   dwdReset
00004628   dwdGenerateSysReset
00004644   IsdwdKeySequenceCorrect
00004678   dwdGetStatus
000046ac   dwdClearFlag
000046bc   dwdGetViolationStatus
00004744   rtiEnableNotification
0000476c   rtiDisableNotification
00004788   rtiGetConfigValue
00004914   muxInit
00004c98   pinmuxGetConfigValue
00004f44   esmInit
00005070   esmError
0000508c   esmEnableError
000050b8   esmDisableError
000050e4   esmTriggerErrorPinReset
000050f4   esmActivateNormalOperation
00005104   esmEnableInterrupt
00005130   esmDisableInterrupt
0000515c   esmSetInterruptLevel
000051e0   esmClearStatus
00005220   esmClearStatusBuffer
0000524c   esmSetCounterPreloadValue
0000526c   esmGetStatus
000052e0   esmGetStatusBuffer
00005340   esmEnterSelfTest
000053b4   esmSelfTestStatus
00005404   esmGetConfigValue
00005564   _coreInitRegisters_
00005670   _coreInitStackPointer_
000056bc   _getCPSRValue_
000056c4   _gotoCPUIdle_
000056dc   _coreEnableVfp_
000056f4   _coreEnableEventBusExport_
0000570c   _coreDisableEventBusExport_
00005724   _coreEnableRamEcc_
0000573c   _coreDisableRamEcc_
00005754   _coreEnableFlashEcc_
00005770   _coreDisableFlashEcc_
00005788   _coreEnableIrqVicOffset_
000057a0   _coreGetDataFault_
000057a8   _coreClearDataFault_
000057bc   _coreGetInstructionFault_
000057c4   _coreClearInstructionFault_
000057d8   _coreGetDataFaultAddress_
000057e0   _coreClearDataFaultAddress_
000057f4   _coreGetInstructionFaultAddress_
000057fc   _coreClearInstructionFaultAddress_
00005810   _coreGetAuxiliaryDataFault_
00005818   _coreClearAuxiliaryDataFault_
0000582c   _coreGetAuxiliaryInstructionFault_
00005834   _coreClearAuxiliaryInstructionFault_
00005848   _disable_interrupt_
00005850   _disable_FIQ_interrupt_
00005858   _disable_IRQ_interrupt_
00005860   _enable_interrupt_
00005868   _esmCcmErrorsClear_
000058f0   _errata_CORTEXR4_57_
00005908   _errata_CORTEXR4_66_
00005920   __TI_PINIT_Base
00005924   __TI_PINIT_Limit
00005928   vimParityErrorHandler
00005bc8   _c_int00
00005e10   esmHighInterrupt
00005f68   esmGroup1Notification
00005f78   esmGroup2Notification
00005f88   memoryPort0TestFailNotification
00005fa4   memoryPort1TestFailNotification
00005fc0   rtiNotification
00006034   canErrorNotification
00006048   canMessageNotification
0000605c   dmaGroupANotification
00006078   _dabort
00006161   __aeabi_memcpy
00006161   __aeabi_memcpy4
00006161   __aeabi_memcpy8
00006161   memcpy
000061fd   __TI_auto_init
000062f0   rtiCompare0Interrupt
0000633d   copy_in
00006385   C$$EXIT
00006389   abort
00006391   exit
000063c8   main
000063f5   _register_unlock
000063fb   _register_lock
00006403   _nop
00006409   __TI_zero_init
0000641b   __TI_decompress_none
00006429   __TI_decompress_rle24
00006430   phantomInterrupt
0000666c   __TI_Handler_Table_Base
00006678   __TI_Handler_Table_Limit
00006680   __TI_CINIT_Base
00006690   __TI_CINIT_Limit
08001500   _lock
08001504   _unlock
08001508   __TI_cleanup_ptr
0800150c   __TI_dtors_ptr
08001510   Tx_Data_CAN
ffffffff   __binit__
ffffffff   __c_args__
ffffffff   binit
UNDEFED    SHT$$INIT_ARRAY$$Base
UNDEFED    SHT$$INIT_ARRAY$$Limit

[201 symbols]
